:100000000C942A001895000018950000189500001F
:10001000189500001895000018950000189500002C
:10002000189500000C94A80618950000189500007B
:10003000189500001895000018950000189500000C
:1000400018950000189500001895000018950000FC
:10005000189500008FE58DBFC4E0E0E84E2E88E0E3
:100060008EBFD8E0F7E05F2EEEEFF7E0A0E6B0E05D
:1000700088278D933197E9F7662481E48ABB81E371
:100080008BBB8FEB87BB8FEB88BB88E084BB83E0A7
:1000900085BB80E081BB8BE382BB80E08FBD81E0CC
:1000A0008EBD8FE181BD87E181BD86E086B980E4A8
:1000B00087B9C398C29AD89ADE9AC498C798C59847
:1000C000F894A8950E94D5078091D300806880930A
:1000D000D300EFEFF1E0A4ECB0E091E00E9436270E
:1000E0000091C400003081E009F080E08F9300911E
:1000F000C4000E3F80E010F009F081E09F91892B51
:10010000882311F40C9487008EEB8093C400009137
:10011000C4004AE0040F01BF89E190E00E94F92584
:10012000EAE0F0E0BB27A0E10E943327013311F49D
:100130000C94E200EAE0F0E0A0E1BB2781E38C93BD
:100140007BE70E942227EBE0F0E0A0E1BB278FE0F5
:100150008C937BE70E942227ECE0F0E001E010E0C6
:10016000A0E1BB277BE70E942427EEE0F0E0A0E1BE
:10017000BB2780E08C937BE70E942227E2E1F0E03E
:1001800000E010E0A0E1BB277BE70E942427EFE01E
:10019000F0E0A0E1BB2780E08C937BE70E94222760
:1001A000E0E1F0E0A0E1BB2780E08C937BE70E94D8
:1001B0002227E1E1F0E0A0E1BB2780E08C937BE720
:1001C0000E942227EBE0F0E0AFEBB0E00E94332783
:1001D0000091BF00043618F011F00C94F1000C945B
:1001E000F40084E68093BF0080E797E9A0ECB0E0DC
:1001F0008D939C93ECE0F0E0AAEBB0E00E943527F1
:10020000EEE0F0E0A5ECB0E00E943327EFE0F0E094
:10021000A6ECB0E00E9433270E94D907E0E1F0E0AD
:10022000AFE6B0E00E943327E1E1F0E0A0E7B0E004
:100230000E943327E2E1F0E0A3E6B0E00E94352718
:10024000A3E6B0E00E94FA24E2E1F0E0A3E6B0E029
:100250007BE70E942427AAEBB0E00D911C910030AF
:1002600050E0150711F00C943B0181E090E0AAEBFF
:10027000B0E08D939C9380E08093D20080916C00DD
:10028000877F80936C0080E08093C80086E0809335
:10029000C2008DE08093C300EBE6F0E0FA93EA93AE
:1002A0000E947716229684E190E00E94F925DE985C
:1002B0000E94E525C49A88EC90E00E94F925A89553
:1002C00081B5886181BD877F81BDE0E6F0E0FA936A
:1002D000EA930E94581B2296A89500916000003076
:1002E00011F40C9479010E94A01A0E949C070C94AE
:1002F0007E0180916C008E7F80936C000E94C91AF1
:1003000084E690E00E94F92500916B00003018F01F
:1003100011F00C948D010C949401EBE6F0E0FA934B
:10032000EA930E94AF1822960027ACE6B0E08C91C9
:1003300080FB0EF401E040E0041711F00C94A201E0
:100340000E94DA0D82E390E00E94F9257894A89546
:1003500081B5886081BD00916F00003011F00C9470
:10036000B70181E090E0AAEBB0E08D939C930091FF
:100370006F00013011F00C94C901AAEBB0E00D91AF
:100380001C9141E050E0040F151FAAEBB0E00D9363
:100390001C93A6EBB0E04D915C91AAEBB0E00D91FF
:1003A0001C910417150718F011F00C94D9010C9446
:1003B000DF0181E090E0AAEBB0E08D939C930027F1
:1003C000ACE6B0E08C9184FB0EF401E041E0041750
:1003D00081E009F080E08F930027ACE6B0E08C91DB
:1003E00080FB0EF401E040E0041781E009F080E0BA
:1003F0009F918923882311F40C941102EAEBF0E019
:10040000FA93EA935A924A9280E0A42DB52D8C93E8
:1004100081E00E94E7240E94D30B249681E00E9491
:10042000E32480E08093BC0080E080936B008091A7
:100430006C008F7780936C000027ACE6B0E08C9165
:1004400080FB0EF401E041E0041711F00C942A0245
:100450000E94D507A895ADE6B0E088278C9300915F
:10046000D200003011F00C941B03E0E6F0E0FA93A8
:10047000EA930E94CF16229600916000003018F097
:1004800011F00C9445020C941B0380916C00806861
:1004900080936C000091D400003011F00C9496020F
:1004A000809160008093C8000027ACE6B0E08C919A
:1004B00084FB0EF401E040E0041711F00C9470028C
:1004C000A0E6B0E08C91AAEBB0E08D9388278C93E6
:1004D000ADE6B0E0E2ECFEE40E943B260C9496020E
:1004E0000027ACE6B0E08C9181FB0EF401E041E026
:1004F000041711F00C949002A0E6B0E00D911127C2
:1005000041E050E0040F151FAAEBB0E00D931C93DF
:10051000ADE6B0E0E2ECFEE40E943B260C949602CD
:10052000ADE6B0E0E4ECFEE40E943B260091D4008E
:10053000023011F00C941B03809160008093C8007E
:1005400000916000013011F00C94B20281E090E063
:10055000AAEBB0E08D939C93ADE6B0E0E2ECFEE454
:100560000E943B2600916000023011F00C940303BE
:10057000A6EBB0E00D911C91013050E0150718F08A
:1005800011F00C94C5020C94FD02A6EBB0E00D91A5
:100590001C9141E050E0041B150BA3E6B0E00D9365
:1005A0001C9301E010E00F931F93A3E6B0E08D9140
:1005B0009C918A939A930E9415252296402F512F41
:1005C0001F910F91040F151FA5E6B0E00D931C932A
:1005D000AAEBB0E04D915C91A5E6B0E00D911C91C5
:1005E0000417150711F40C94D102A5E6B0E08D9123
:1005F0009C91AAEBB0E08D939C93ADE6B0E0E2EC69
:10060000FEE40E943B2600916000033011F00C9440
:100610000F03ADE6B0E0E4ECFEE40E943B2600915F
:100620006000043011F00C941B03ADE6B0E0E6EC82
:10063000FEE40E943B260027ACE6B0E08C9184FBF0
:100640000EF401E041E0041781E009F080E08F93AF
:100650000027ACE6B0E08C9181FB0EF401E041E0B4
:10066000041781E009F080E09F9189238F93009126
:10067000D200013081E009F080E09F918923882336
:1006800011F40C948603AAEBB0E00D911C9101309B
:1006900050E0150711F00C948603E0E6F0E0FA93C1
:1006A000EA930E94CF16229600916000003080E00D
:1006B00010F009F081E08F93A6EBB0E04D915C91D2
:1006C000A0E6B0E00D9111270417150781E008F0AE
:1006D00080E09F918923882311F40C948603A0E67F
:1006E000B0E00D91112741E050E0040F151FAAEB77
:1006F000B0E00D931C93ADE6B0E0E2ECFEE40E94A6
:100700003B2680916C00806880936C00EBE6F0E003
:10071000FA93EA930E947716229600916B000430B8
:1007200011F00C949A030E948D0780916C008068F0
:1007300080936C0000916B00013011F00C94AB03BE
:10074000ADE6B0E0E4ECFEE40E943B2680916C0054
:10075000806880936C0080E08093600000916B0063
:10076000023081E009F080E08F930091BF000436F1
:1007700081E008F080E09F918923882311F40C9494
:10078000C903AFEBB0E08C918B5F8C9381E08093D9
:10079000600000916B00033081E009F080E08F93EE
:1007A0000091BF00053081E009F080E09F9189232E
:1007B000882311F40C94E20381E08093BF0081E070
:1007C0008093600000916B00033081E009F080E0CD
:1007D0008F930091BF00053080E010F009F081E0B8
:1007E0009F918923882311F40C94FE03AFEBB0E0B2
:1007F0008C9185508C9381E0809360000091600023
:10080000013011F00C942B048EB5887F8EBD5A9266
:100810004A928091BF00A42DB52D8C9381E00E9457
:10082000E7240E946521229681E00E94E324EBE008
:10083000F0E0AFEBB0E07BE70E9422270091D2000E
:10084000013011F00C94260481E08EBD80916C0083
:10085000806880936C00EDE6F0E0ADE6B0E00E94C9
:100860004526ADE6B0E08C91803081E009F480E06F
:100870008F9300916B00003081E009F480E09F913C
:10088000892B8F930091BC00013081E009F080E05A
:100890009F91892B882311F40C941C020091BC00B9
:1008A000013011F00C94750480E08093BC00ADE63B
:1008B000B0E0E4ECFEE40E943B260027ACE6B0E0AA
:1008C0008C9181FB0EF401E041E0041711F00C94CF
:1008D000750481E090E0AAEBB0E08D939C93ADE6C7
:1008E000B0E0E2ECFEE40E943B26ADE6B0E0E2ECD4
:1008F000FEE40E944D2711F00C94E7040091D20011
:10090000013011F00C9486040E948D07A6EBB0E034
:100910004D915C91AAEBB0E00D911C910417150765
:1009200018F011F00C94E2040027ACE6B0E08C91D2
:1009300080FB0EF401E040E0041711F00C94B304C6
:10094000EAEBF0E0FA93EA935A924A9280E0A42DFF
:10095000B52D8C9381E00E94E7240E94D30B24964E
:1009600081E00E94E3240027ACE6B0E08C9180FB9C
:100970000EF401E041E0041711F00C94E0040E9431
:100980009C070027ACE6B0E08C9180FB0EF401E000
:1009900040E0041711F00C94E004EAEBF0E0FA9365
:1009A000EA935A924A9280E0A42DB52D8C9381E06F
:1009B0000E94E7240E94D30B249681E00E94E32446
:1009C0000C94E50480E08093C8000C941506E4ECD8
:1009D000FEE40E944D2711F00C947F050091D20097
:1009E000013011F00C94F6040E948D07AAEBB0E0E0
:1009F0000E94FA240027A3EDB0E08C9187FB0EF44F
:100A000001E041E0041711F00C941B050027ACE64F
:100A1000B0E08C9184FB0EF401E040E0041711F08B
:100A20000C941605AAEBB0E00E9401258091D3003A
:100A30008F778093D300A6EBB0E04D915C91AAEB49
:100A4000B0E00D911C910417150718F011F00C94EB
:100A50002B050C94310581E090E0AAEBB0E08D937A
:100A60009C930027ACE6B0E08C9180FB0EF401E093
:100A700040E0041711F00C945005EAEBF0E0FA9313
:100A8000EA935A924A9280E0A42DB52D8C9381E08E
:100A90000E94E7240E94D30B249681E00E94E32465
:100AA0000027ACE6B0E08C9180FB0EF401E041E061
:100AB000041711F00C947D050E949C070027ACE6FA
:100AC000B0E08C9180FB0EF401E040E0041711F0DF
:100AD0000C947D05EAEBF0E0FA93EA935A924A927D
:100AE00080E0A42DB52D8C9381E00E94E7240E9424
:100AF000D30B249681E00E94E3240C941506E6ECC7
:100B0000FEE40E944D2711F00C94F7050091D200ED
:100B1000013011F00C948E050E948D07AAEBB0E015
:100B20000D911C91013050E0150718F011F00C9454
:100B30009B050C94A105AAEBB0E00E9401250C9442
:100B4000A905A6EBB0E08D919C91AAEBB0E08D9346
:100B50009C930027ACE6B0E08C9180FB0EF401E0A2
:100B600040E0041711F00C94C805EAEBF0E0FA93AA
:100B7000EA935A924A9280E0A42DB52D8C9381E09D
:100B80000E94E7240E94D30B249681E00E94E32474
:100B90000027ACE6B0E08C9180FB0EF401E041E070
:100BA000041711F00C94F5050E949C070027ACE691
:100BB000B0E08C9180FB0EF401E040E0041711F0EE
:100BC0000C94F505EAEBF0E0FA93EA935A924A9214
:100BD00080E0A42DB52D8C9381E00E94E7240E9433
:100BE000D30B249681E00E94E3240C941506E8ECD4
:100BF000FEE40E944D2711F00C9405060E948D071B
:100C000080E08093C8000C941506EAECFEE40E9494
:100C10004D2711F00C941506ECE0F0E0AAEBB0E0E3
:100C20007BE70E9424270C94150681E090E00E9447
:100C3000F9250027ACE6B0E08C9187FB0EF401E0CB
:100C400040E0041718F011F00C9428060C94A60646
:100C500000916B00003018F011F00C9431060C94E8
:100C60009806A895E0E6F0E0FA93EA930E947716DA
:100C7000229600916000043011F00C948C060E94C2
:100C80008D0780E08093C8000E94D70785E090E040
:100C90000E94F92580E080936200E0E6F0E0FA939C
:100CA000EA930E9477162296A2E6B0E08C918F5FBD
:100CB0008C9388E090E00E94F9250091600000305C
:100CC00081E009F080E08F9300916200043680E0BB
:100CD00010F009F081E09F91892B882311F40C9486
:100CE0004D0600916200043618F011F00C947A065B
:100CF0000C94890681B5886181BD877F81BDE3E65B
:100D0000F0E0FA93EA930E944B08229681B588603E
:100D100081BD80E08093600081E090E00E94F92531
:100D200000916000003011F00C9431060C949C0688
:100D30008AE090E00E94F9250091D200003011F085
:100D40000C94A60685E090E00E94F9250C94170209
:100D50000F921F922F923F924F925F927F92AF928B
:100D6000BF920F931F932F933F934F935F936F9374
:100D70007F938F939F93AF93BF93CF93DF93EF9323
:100D8000FF938FB78F93F89489B78B7F89BF8EB508
:100D9000887F8EBD5A924A9280E092E0A42DB52DB4
:100DA0008D939C9382E00E94E7240E946124229606
:100DB00082E00E94E3240091DD000A3011F00C94DF
:100DC000E3060E94D5070E94E51D0091DD000A3070
:100DD00011F00C94F0060E94D70780E08093DD00AC
:100DE000ADEDB0E08C918F5F8C93A8950027ACE6B9
:100DF000B0E08C9180FB0EF401E040E0041711F0AC
:100E00000C9415075A924A9280E092E0A42DB52DD9
:100E10008D939C9382E00E94E7240E946124229695
:100E200082E00E94E3240E94E51DA9EDB0E04D910F
:100E30005D916D917C91A5EDB0E00D911D912D918D
:100E40003C910E94992680E00CF481E08F9300276A
:100E5000ACE6B0E08C9180FB0EF401E040E00417BA
:100E600081E009F080E09F918923882311F40C949C
:100E7000460780E49CE990934D0080934C0081E00C
:100E80008EBD89B7846089BF0C946F0780E0809322
:100E9000D20080916C00877F80936C000027ACE6C5
:100EA000B0E08C9180FB0EF401E040E0041711F0FB
:100EB0000C946307ACE6B0E08C9184FBACEBB0E043
:100EC000882780F98C930091C5004FE70423A1E6A1
:100ED000B0E00C930E94D70780E08093C8008F9108
:100EE0008FBFFF91EF91DF91CF91BF91AF919F9114
:100EF0008F917F916F915F914F913F912F911F91B2
:100F00000F91BF90AF907F905F904F903F902F9048
:100F10001F900F901895F894FFCF89B78B7F89BFEA
:100F20008EB5887F8EBD80E08093D20080916C006A
:100F3000877F80936C000895DE9A6E98C498C59858
:100F4000C7980E94D707E2E0F0E00E947025DE9883
:100F5000C49A0E94E52584E690E00E94F925A895B0
:100F600080916C008E7F80936C00E0E6F0E0FA9355
:100F7000EA930E94581B229600916000003011F401
:100F80000C94D20780916C00816080936C0084E6A1
:100F900090E00E94F925DE9A6E98C498C598C7988B
:100FA0000C94D4070E94DA0D0895AB980895AB9A7B
:100FB000089581E00E94082680916C008F7E8093C6
:100FC0006C000091C50041E00423A881B9810C9315
:100FD000A881B9810C91003011F40C94F407809130
:100FE0006C00806180936C0080916C008D7F809399
:100FF0006C000091C50042E00423A881B9810C93E4
:10100000A881B9810C91003011F40C940C088091E6
:101010006C00826080936C0080916C008F7D809367
:101020006C000091C50040E20423A881B9810C93B3
:10103000A881B9810C91003011F40C94240880919E
:101040006C00806280936C008091D3008F7B8093D2
:10105000D3000091C60046E00423A881B9810C9317
:10106000A881B9810C9142E00E943D270C93A88190
:10107000B9818C918093D4000091D400033011F099
:101080000C94450882E08093D40081E0481A8827B8
:10109000580A2296089582E00E94082681E00E9464
:1010A000082681E00E94082680E0AA81BB818C93FB
:1010B00083E4A0EAB0E08C938FE4A1EAB0E08C93E3
:1010C0008EE4A2EAB0E08C9386E4A3EAB0E08C93CD
:1010D00089E4A4EAB0E08C93ACE6B0E08C9185FBA7
:1010E000A881B981882780F98C9380916C008062F7
:1010F00080936C00A6E7B0E00D911D912D913C917D
:10110000A6E9B0E00D931D932D933C935A924A9219
:10111000A6E9B0E00D911D912D913C91A42DB52D26
:101120000D931D932D933C9384E00E94E7245A92E3
:101130004A9280E090E0A42DB52D8D939C9382E09F
:101140000E94E7245A924A9281E0A42DB52D8C93F7
:1011500081E00E94E7240E94E90E269687E00E9423
:10116000E3248FE00E940826E8EAF0E006E0A88188
:10117000B9810E941427A881B981ECECFEE40E9499
:101180004D270FB68FE0481A8827580A22960FBEBF
:1011900081E009F080E08F9300919100003181E0BF
:1011A00009F080E09F918923882311F40C9426098B
:1011B00081E0AA81BB818C93A6E9B0E00D911D91DD
:1011C0002D913C91A6E7B0E00D931D932D933C9398
:1011D00080916C008F7D80936C005A924A92A6E9B0
:1011E000B0E00D911D912D913C91A42DB52D0D9345
:1011F0001D932D933C9384E00E94E7245A924A92D7
:1012000080E090E0A42DB52D8D939C9382E00E9408
:10121000E7245A924A9280E0A42DB52D8C9381E068
:101220000E94E7240E94E90E269687E00E94E324AC
:10123000A6E9B0E00D911D912D913C91A6E7B0E09B
:101240000D931D932D933C930E948009A881B98131
:101250008C9180FBACE6B0E08C9185F98C93AAE789
:10126000B0E00D911D912D913C91A6E7B0E00D935A
:101270001D932D933C93A6E7B0E00D911D912D9108
:101280003C91A6E9B0E00D931D932D933C935A92A7
:101290004A92A6E9B0E00D911D912D913C91A42DAB
:1012A000B52D0D931D932D933C9384E00E94E7246C
:1012B0005A924A9280E090E0A42DB52D8D939C9394
:1012C00082E00E94E7245A924A9280E0A42DB52D34
:1012D0008C9381E00E94E7240E94E90E269687E025
:1012E0000E94E324AA81BB818C91AE81BF818D9342
:1012F00088278C9384E0481A8827580A26960895F0
:1013000082E00E94082681E00E94082681E00E9477
:101310000826789481E090E0AC81BD818D939C9308
:10132000EA81FB81FA93EA93EE81FF81FA93EA93D3
:101330000E94960B2496AA81BB810C91013011F07A
:101340000C94AD0982E090E0AC81BD818D939C93BB
:1013500081E08093C5000C94C909023011F00C940F
:10136000BC0983E090E0AC81BD818D939C9380E0CB
:101370008093C5000C94C909033011F00C94C9097D
:1013800084E090E0AC81BD818D939C9383E0809359
:10139000C500EEE0F0E0A5ECB0E07BE70E9422277C
:1013A000EC81FD81FA93EA935A924A9280E0A42D4F
:1013B000B52D8C9381E00E94E7240E94D30B2496E4
:1013C00081E00E94E3240091D200003011F00C94DF
:1013D000E30988EC90E00E94F92585E090E0AC817B
:1013E000BD818D939C93EA81FB81FA93EA93EE8110
:1013F000FF81FA93EA930E94960B2496EEE0F0E0C8
:10140000A5ECB0E00E943327AA81BB810C91033088
:1014100011F00C940D0A0C94AA0AAA81BB810C91BC
:10142000013011F00C941B0AA5ECB0E08C9188609F
:101430008C930C94240A023011F00C94240AA5EC2D
:10144000B0E08C91877F8C93EEE0F0E0A5ECB0E00B
:101450007BE70E94222788EC90E00E94F92586E035
:1014600090E0AC81BD818D939C93EA81FB81FA93DE
:10147000EA93EE81FF81FA93EA930E94960B2496F9
:10148000AA81BB810C91033011F00C94490A0C9491
:10149000AA0AEEE0F0E0A5ECB0E00E943327AA81B2
:1014A000BB810C91013011F00C945D0AA5ECB0E009
:1014B0008C9184608C930C94660A023011F00C9429
:1014C000660AA5ECB0E08C918B7F8C93EEE0F0E0A7
:1014D000A5ECB0E07BE70E94222788EC90E00E9418
:1014E000F92587E090E0AC81BD818D939C93EA81E2
:1014F000FB81FA93EA93EE81FF81FA93EA930E94CB
:10150000960B2496EEE0F0E0A5ECB0E00E943327C5
:10151000AA81BB810C91013011F00C94960AA5ECC4
:10152000B0E08C9180628C930C949F0A023011F091
:101530000C949F0AA5ECB0E08C918F7D8C93EEE02B
:10154000F0E0A5ECB0E07BE70E94222788EC90E079
:101550000E94F92588E090E0AC81BD818D939C9339
:10156000EC81FD81FA93EA930E94740B229600911C
:10157000C50043E00423A881B9810C93A881B981F7
:101580000C91003011F00C94CD0A83E090E0AC8116
:10159000BD818D939C930C94E30A013011F00C945F
:1015A000D90A82E090E0AC81BD818D939C930C942C
:1015B000E30A033011F00C94E30A84E090E0AC817C
:1015C000BD818D939C93EC81FD81FA93EA930E94F7
:1015D000740B22960091C50048E00423A881B981CC
:1015E0000C93A881B9810C91003011F00C94000B80
:1015F0008AE090E0AC81BD818D939C930C940A0BA2
:10160000083011F00C940A0B89E090E0AC81BD81A8
:101610008D939C93EC81FD81FA93EA930E94740B65
:1016200022960091C50044E00423A881B9810C935F
:10163000A881B9810C91003011F00C94270B8BE03C
:1016400090E0AC81BD818D939C930C94310B043060
:1016500011F00C94310B8CE090E0AC81BD818D9346
:101660009C93EC81FD81FA93EA930E94740B22967D
:101670000091C50040E20423A881B9810C93A881A0
:10168000B9810C91003011F00C944E0B8DE090E07C
:10169000AC81BD818D939C930C94580B003211F05A
:1016A0000C94580B8EE090E0AC81BD818D939C939F
:1016B000EC81FD81FA93EA930E94740B22968FE0ED
:1016C00090E0AC81BD818D939C93EC81FD81FA9378
:1016D000EA930E94740B22960E94D90784E0481A6C
:1016E0008827580A26960895E881F981FA93EA93A3
:1016F0005A924A9280E0A42DB52D8C9381E00E94ED
:10170000E7240E94D30B249681E00E94E32482E325
:1017100090E00E94F9250091D200003011F00C9465
:101720008B0B82E390E00E94F925089581E00E94EE
:101730000826EA81FB81FA93EA935A924A9280E062
:10174000A42DB52D8C9381E00E94E7240E94D30B39
:10175000249681E00E94E32484E690E00E94F9252B
:10176000E881F981FA93EA930E9477162296A8817C
:10177000B9810C91003018F011F00C94C10B0C944D
:10178000B00B0E948D0784E190E00E94F925A881AA
:10179000B9818C91AC81BD818C9381E0481A8827F6
:1017A000580A2296089582E00E94082681E00E944D
:1017B00008268EB5887F8EBD80916C00877F8093D0
:1017C0006C00A6E7B0E00D911D912D913C91A6E92A
:1017D000B0E00D931D932D933C935A924A92A6E943
:1017E000B0E00D911D912D913C91A42DB52D0D933F
:1017F0001D932D933C9384E00E94E7245A924A92D1
:10180000AA85BB858D919C91A42DB52D8D939C931C
:1018100082E00E94E7245A924A9280E0A42DB52DDE
:101820008C9381E00E94E7240E94E90E269687E0CF
:101830000E94E32440E050E060E070E0A2E9B0E004
:101840000D911D912D913C910E94992611F00C94BF
:101850002B0C0C94D40D0E9419215A924A9280911B
:10186000BF00A42DB52D8C9381E00E94E7240E9437
:101870006521229681E00E94E3245A924A92A0ECCC
:10188000B0E08D919C91A42DB52D8D939C9382E019
:101890000E94E7240E94FD21229682E00E94E32418
:1018A000A6E9B0E00D911D912D913C91A5EDB0E020
:1018B0000D931D932D933C93A6E9B0E00D911D91DE
:1018C0002D913C91A2E9B0E04D915D916D917C919B
:1018D0000E948F26A9EDB0E00D931D932D933D93AB
:1018E00080E0A881B9818C930E94E51D81E090E0A1
:1018F000AA81BB818D939C93AA81BB810D911C9180
:101900000F3F51E0150718F011F00C94B60CAA81A6
:10191000BB81AD90BC90ADEDB0E0AA0DBB1D0C91AC
:101920000F3F81E009F080E08F93AA81BB81AD90E9
:10193000BC90AEEDB0E0AA0DBB1D0C910F3E80E057
:1019400010F009F081E09F918923882311F40C9411
:10195000AF0C81E0A881B9818C930C94B60CAA815C
:10196000BB810E94FA2410F40C947C0CA881B981EC
:101970000C91013011F00C94740CAA81BB81AD90D4
:10198000BC90AFEDB0E0AA0DBB1D8C91AA81BB81CC
:101990008D9388278C93AA81BB810D911C9140E186
:1019A00050E00E944F25AA81BB814D935C9380E15A
:1019B0008093C700AA81BB810D911C91013050E03A
:1019C000150711F00C94E90C84E08093C7000C9487
:1019D000760D023050E0150711F00C94F40C85E000
:1019E0008093C7000C94760D033050E0150711F07A
:1019F0000C94FF0C86E08093C7000C94760D0430A5
:101A000050E0150711F00C940A0D87E08093C70091
:101A10000C94760D053050E0150711F00C94150D5F
:101A200088E08093C7000C94760D063050E01507CF
:101A300011F00C94200D8AE08093C7000C94760D71
:101A4000073050E0150711F00C942B0D8CE08093BB
:101A5000C7000C94760D083050E0150711F00C9477
:101A6000360D8EE08093C7000C94760D093050E05F
:101A7000150711F00C94410D80E18093C7000C9480
:101A8000760D0A3050E0150711F00C944C0D84E1EE
:101A90008093C7000C94760D0B3050E0150711F0C1
:101AA0000C94570D88E18093C7000C94760D0C3090
:101AB00050E0150711F00C94620D8CE18093C70083
:101AC0000C94760D0D3050E0150711F00C946D0D4F
:101AD00080E28093C7000C94760D0E3050E015071D
:101AE00011F00C94760D88E28093C700A2E9B0E073
:101AF0000D911D912D913C9140E052E060E070E02D
:101B00000E941826A7E6B0E00D931D932D933D93F8
:101B1000A7E6B0E00D911D912D913C91A7ECB0E0AE
:101B20004C915527662777270E947925A7E6B0E0D4
:101B30004D935D936D937D93A7E6B0E00D911D915C
:101B40002D913C9148EE53E060E070E00E947925D1
:101B5000A7E6B0E04D935D936D937D93AC81BD811D
:101B60000C91003011F00C94D40D00916F000130F5
:101B700011F00C94C20DECE0F0E0AAEBB0E07BE7D2
:101B80000E94242781E08093D20088EC9FEA909302
:101B90004D0080934C0089B7846089BF81E08EBD81
:101BA00085E090E00E94F92583E0481A8827580ACA
:101BB00024960895A895A6E7B0E00D911D912D916A
:101BC0003C91AAE7B0E00D931D932D933C93A6E7BB
:101BD000B0E00D911D912D913C91A6E9B0E00D93DF
:101BE0001D932D933C935A924A92A6E9B0E00D9131
:101BF0001D912D913C91A42DB52D0D931D932D93E9
:101C00003C9384E00E94E7245A924A9280E090E05C
:101C1000A42DB52D8D939C9382E00E94E7245A92C7
:101C20004A9280E0A42DB52D8C9381E00E94E72498
:101C30000E94E90E269687E00E94E324A895A6EB71
:101C4000B0E00D911C91013050E0150710F00C949C
:101C5000500E5A924A9281E0A42DB52D8C9381E0CA
:101C60000E94E7240E945722229681E00E94E324EA
:101C70008CE291E00E94F9255A924A9280E0A42DCC
:101C8000B52D8C9381E00E94E7240E945722229672
:101C900081E00E94E32480916C00816080936C005D
:101CA000A895A6E7B0E00D911D912D913C91A6E974
:101CB000B0E00D931D932D933C93AAEBB0E00D91F2
:101CC0001C91003050E0150781E009F080E08F930F
:101CD000A6EBB0E04D915C91AAEBB0E00D911C91A8
:101CE0000417150780E010F009F081E09F91892B1F
:101CF000882311F40C94820E81E090E0AAEBB0E00E
:101D00008D939C930E94D707089584E00E94082633
:101D1000A5EDB0E00D911D912D913C91A881B98167
:101D20000D931D932D933C93A6E7B0E00D911D916B
:101D30002D913C91A6E9B0E00D931D932D933C931A
:101D40005A924A92A6E9B0E00D911D912D913C91D5
:101D5000A42DB52D0D931D932D933C9384E00E94EB
:101D6000E7245A924A928FE19EE4A42DB52D8D93DB
:101D70009C9382E00E94E7245A924A9280E0A42D2C
:101D8000B52D8C9381E00E94E7240E94E90E2696EF
:101D900087E00E94E324A6E7B0E00D911D912D910C
:101DA0003C91A6E9B0E00D931D932D933C93A8813F
:101DB000B9810D911D912D913C91A5EDB0E00D9350
:101DC0001D932D933C9384E0481A8827580A229645
:101DD000089581E00E94082681E00E94082681E0A3
:101DE0000E94082680E090E0A8EBB0E08D939C93E1
:101DF00080916C008F7B80936C0000E010E020E00D
:101E000030E0A2E9B0E00D931D932D933C930027A1
:101E1000ACE6B0E08C9185FB0EF401E041E00417E4
:101E200081E009F080E08F93A885B9850D911C9120
:101E3000003050E0150781E009F480E09F9189238C
:101E40008F93AE81BF810C91003081E009F080E07A
:101E50009F918923882311F40C94890FAAE9B0E09B
:101E6000E885F9850E94AC26EAE9F0E0A8E6B7E04B
:101E70000E940827E8E6F7E0AAE9B0E01127222748
:101E800004E033270E94512681E4AC81BD818C930C
:101E9000AC81BD818C918093A00081E0EAE9F0E003
:101EA00001E00A93ADE6B0E00E940D27ADE6B0E098
:101EB0008C91A1EAB0E08C9382E0EAE9F0E001E0E5
:101EC0000A93ADE6B0E00E940D27ADE6B0E08C913C
:101ED000A2EAB0E08C9383E0EAE9F0E001E00A9343
:101EE000ADE6B0E00E940D27ADE6B0E08C91A3EA2C
:101EF000B0E08C9384E0EAE9F0E001E00A93ADE61B
:101F0000B0E00E940D27ADE6B0E08C91A4EAB0E00D
:101F10008C9389B78B7F89BF8EB5887F8EBD81B545
:101F2000886181BD877F81BDAEECB0E00D911D91D0
:101F30002D913C91AAECB0E00D931D932D933C9311
:101F4000AAE7B0E04D915D916D917C91A6E7B0E07C
:101F50000D911D912D913C910E94992611F00C94A8
:101F6000BB0F02E010E020E030E0AAECB0E00D93FF
:101F70001D932D933C9380E0A881B9818C93EA81D5
:101F8000FB81FA93EA935A924A92AE85BF850D91EE
:101F90001D912D913C91A42DB52D0D931D932D9345
:101FA0003C9384E00E94E7240E94AE1F249684E0C4
:101FB0000E94E324AA81BB810C910E3F11F40C9482
:101FC000ED0F80916C00816080936C0080916C00BB
:101FD000806480936C000C9400105A924A92AA85F7
:101FE000BB858D919C91A42DB52D8D939C9382E002
:101FF0000E94E7240E940311229682E00E94E324BB
:10200000A881B9818C918F5F8C9340917300A881D6
:10201000B9810C91041781E009F080E08F930027CB
:10202000ACE6B0E08C9186FB0EF401E041E00417D1
:1020300081E009F480E09F918923882311F40C94B6
:10204000B610009182000B3011F00C946310EAEC92
:10205000F0E0FA93EA935A924A92AAECB0E00D911A
:102060001D912D913C91A42DB52D0D931D932D9374
:102070003C9384E00E94E7240E941B15249684E090
:102080000E94E324EA85FB85FA93EA935A924A92E6
:10209000AAECB0E00D911D912D913C91A42DB52D90
:1020A0000D931D932D933C9384E00E94E7240E949E
:1020B000B114249684E00E94E32480E0A881B981D1
:1020C0008C930C94B410AAE7B0E04D915D916D91A2
:1020D0007C91A6E7B0E00D911D912D913C910E945D
:1020E000992611F00C947A10AA85BB850E94EB24E6
:1020F0000C94B410EAECF0E0FA93EA935A924A9204
:10210000AAECB0E00D911D912D913C91A42DB52D1F
:102110000D931D932D933C9384E00E94E7240E942D
:102120001B15249684E00E94E324EA85FB85FA933C
:10213000EA935A924A92AAECB0E00D911D912D912A
:102140003C91A42DB52D0D931D932D933C9384E0CC
:102150000E94E7240E94B114249684E00E94E324A4
:1021600080E0A881B9818C930C94BA10AA85BB85B4
:102170000E94EB240027ACE6B0E08C9186FB0EF4C5
:1021800001E041E0041711F00C94BF0FC49AA88538
:10219000B9850D911C91003050E0150711F00C9499
:1021A000D910A8EBB0E08D919C91A6EBB0E08D9397
:1021B0009C930091D200013081E009F080E08F9380
:1021C0000027ACE6B0E08C9180FB0EF401E040E02B
:1021D000041781E009F080E09F918923882311F49E
:1021E0000C94FD1080E593EC90934D0080934C008F
:1021F00081E08EBD89B7846089BF83E0481A882753
:10220000580A2696089584E00E94082684E00E94D9
:10221000082681E00E94082681E00E94082681E0CD
:102220000E94082681E00E94082680E0AE81BF81DE
:102230008C93AE81BF810C910F3018F011F00C948B
:10224000BE1281E0AC81BD818C93AC81BD810C91CB
:102250000C3018F011F00C9445118FEF0E94EC2512
:102260000E94EE250E94ED25AC81BD81AD90BB247E
:10227000A4E8B0E0AA0DBB1D8C93AC81BD818C910C
:102280008F5F8C9310F40C9425118DE0AC81BD818F
:102290008C93AC81BD810C91043118F011F00C9439
:1022A00063118FEF0E94EC250E94EE250E94ED2520
:1022B000A881B9818C93AC81BD818C918F5F8C9307
:1022C00010F40C944911EA85FB85FA93EA93EA85A8
:1022D000FB85FA93EA930E94461324960027ACE606
:1022E000B0E08C9186FB0EF401E041E0041711F0A0
:1022F0000C947C110C94B61280E0AA81BB818C9363
:1023000000919000003281E009F080E08F9300910D
:102310009000003181E009F080E09F91892B8823B3
:1023200011F40C94971181E0AA81BB818C930091E8
:102330008500003081E009F480E08F9300918500F2
:10234000053E81E009F480E09F9189238F93AA8163
:10235000BB810C91013081E009F080E09F918923DD
:10236000882311F40C94AB1200919000003211F00C
:102370000C94BE11A8EBB0E00E94FA240027ACE652
:10238000B0E08C9185FB0EF401E040E0041711F001
:102390000C94F31181E0AC81BD818C93AC85BD853B
:1023A0004D915C91A8EBB0E00D911C9104171507BD
:1023B00081E009F080E08F93A8EBB0E00D911C91D3
:1023C000003050E0150780E010F009F081E09F91A7
:1023D0008923882311F40C94F11180E0AC81BD8134
:1023E0008C930C94271280E0AC81BD818C9381E0AA
:1023F000A881B9818C93A881B9810C91053018F01E
:1024000011F00C942712A881B981AD90BB24AFE9DB
:10241000B0E0AA0DBB1D4C91A881B981AD90BB2441
:10242000A4E8B0E0AA0DBB1D0C91041711F40C94A4
:102430001F1281E0AC81BD818C930C942712A8817E
:10244000B9818C918F5F8C9310F40C94FB11AC814B
:10245000BD810C91003081E009F080E08F93AC8564
:10246000BD850D911C910F315EE4150781E009F0E7
:1024700080E09F91892B882311F40C94AB120E9469
:10248000D812A885B9850D911D912D913C9140E000
:1024900052E060E070E00E947925A2E9B0E04D933F
:1024A0005D936D937D93E6E9F0E0FA93EA935A9297
:1024B0004A92AE85BF850D911D912D913C91A42D21
:1024C000B52D0D931D932D933C9384E00E94E7243A
:1024D0000E94B114249684E00E94E324809190002D
:1024E00080939100AC85BD850D911C910F315EE408
:1024F000150711F00C947C12AC81BD810C91003059
:1025000011F00C94AB1280916C00806480936C008D
:1025100000919100003181E009F080E08F93AC855B
:10252000BD850D911C910F315EE4150781E009F422
:1025300080E09F918923882311F40C94AB12AA8523
:10254000BB850D911D912D913C91AEECB0E00D93AA
:102550001D932D933C9300918500003011F00C9455
:10256000B61280916C00806480936C00AE81BF8154
:102570008C918F5F8C9310F40C9419118FEF0E9443
:10258000EC250E94EE250E94ED25A0E6B0E08C939C
:102590008FEF0E94EC250E94EE250E94ED25A0E61B
:1025A000B0E08C938CE0481A8827580A2C9608953E
:1025B00081E00E940826A8EAB0E088278C9381E099
:1025C000A881B9818C93A881B9810C91083018F049
:1025D00011F00C941213A881B981AD90BB24A4E82A
:1025E000B0E0AA0DBB1D0C91003211F40C940A133B
:1025F000A881B981AD90BB24A4E8B0E0AA0DBB1DB1
:102600008C91A8EAB0E08F930E9469258F918D93F9
:1026100088278C93A881B9818C918F5F8C9310F45B
:102620000C94E312A8EAB0E00E946925E4EDFEE410
:102630000E943B2689E0A881B9818C93A881B98149
:102640000C910B3018F011F00C944013A881B98153
:10265000AD90BB24A4E8B0E0AA0DBB1D8C91A8EA04
:10266000B0E08F930E9469258F918D9388278C937A
:10267000A881B9818C918F5F8C9310F40C941E13F8
:1026800081E0481A8827580A2296089581E00E941E
:10269000082681E00E94082684E00E9408268FEF29
:1026A0000E94EC250E94EE250E94ED25AC81BD81A3
:1026B0008C938FEF0E94EC250E94EE250E94ED2561
:1026C000AA81BB818C93AA81BB810C9111272227FF
:1026D000332740E051E060E070E00E941826A885B2
:1026E000B9850D931D932D933D93A885B9850D91C3
:1026F0001D912D913C91AC81BD814C915527662750
:1027000077270E948F26A885B9850D931D932D9359
:102710003D93A885B9850D911D912D913C9140E087
:1027200050E061E070E00E941826A881B9810D9305
:102730001D932D933D938FEF0E94EC250E94EE2573
:102740000E94ED25AC81BD818C938FEF0E94EC251A
:102750000E94EE250E94ED25AC81BD818C938FEF08
:102760000E94EC250E94EE250E94ED25AC81BD81E2
:102770008C938FEF0E94EC250E94EE250E94ED25A0
:10278000AC81BD818C938FEF0E94EC250E94EE25D9
:102790000E94ED25AC81BD818C938FEF0E94EC25CA
:1027A0000E94EE250E94ED25AA81BB818C93AA810F
:1027B000BB810C9111272227332740E051E060E0D4
:1027C00070E00E941826A885B9850D931D932D935E
:1027D0003D93A885B9850D911D912D913C91AC81BA
:1027E000BD814C915527662777270E948F26A885A3
:1027F000B9850D931D932D933D93A885B9850D91B2
:102800001D912D913C91A881B9814D915D916D9162
:102810007C910E948F26A885B9850D931D932D93D9
:102820003D938FEF0E94EC250E94EE250E94ED253E
:10283000AC81BD818C938FEF0E94EC250E94EE2528
:102840000E94ED25AA81BB818C93AA81BB810C914A
:1028500011272227332740E051E060E070E00E941A
:102860001826A881B9810D931D932D933D93A881BE
:10287000B9810D911D912D913C91AC81BD814C91FF
:102880005527662777270E948F26A881B9810D9347
:102890001D932D933D938FEF0E94EC250E94EE2512
:1028A0000E94ED25AC81BD818C938FEF0E94EC25B9
:1028B0000E94EE250E94ED25AA81BB818C93AA81FE
:1028C000BB810C9111272227332740E051E060E0C3
:1028D00070E00E941826AE81BF810D931D932D9349
:1028E0003D93AE81BF810D911D912D913C91AC81A5
:1028F000BD814C915527662777270E948F26AE8190
:10290000BF810D931D932D933D93AE81BF810D919A
:102910001D912D913C9140E050E061E070E00E94FB
:102920001826AE81BF810D931D932D933D93AE81EB
:10293000BF810D911D912D913C91A881B9814D913F
:102940005D916D917C910E948F26AE81BF810D9328
:102950001D932D933D9386E0481A8827580A2696A2
:10296000089584E00E94082684E00E940826AC8135
:10297000BD810D911D912D913C9142E050E060E0B0
:1029800070E00E949426A881B9810D931D932D9328
:102990003D93A3E7B0E00C91112722273327A881AC
:1029A000B9814D915D916D917C910E941826AA810B
:1029B000BB810D931D932D933D93AA81BB810D91F6
:1029C0001D912D913C91AAE7B0E04D915D916D91E3
:1029D0007C910E948F26AA81BB810D931D932D931C
:1029E0003D93009182000B3011F40C940915AA81DB
:1029F000BB810D911D912D913C9140E250E060E032
:102A000070E00E948F26AA81BB810D931D932D93A8
:102A10003D93AA81BB810D911D912D913C91AE8179
:102A2000BF810D931D932D933C9388E0481A88270E
:102A3000580A2496089584E00E94082682E00E94A5
:102A40000826009182000B3011F00C945F15AC81C8
:102A5000BD810D911D912D913C9140E850E060E0C9
:102A600070E00E947925A5EDB0E04D935D936D93E4
:102A70007D93AC81BD810D911C9140E850E00E9496
:102A80004F25A881B9810D931C93A881B9810D911F
:102A90001C9144E050E00E940E26A881B9810D935C
:102AA0001C93A881B9810D911C9144E050E0040F62
:102AB000151FA881B9810D931C930C949515AC81B9
:102AC000BD810D911D912D913C9140E051E060E060
:102AD00070E00E947925A5EDB0E04D935D936D9374
:102AE0007D93AC81BD810D911C9140E051E00E942D
:102AF0004F25A881B9810D931C93A881B9810D91AF
:102B00001C9142E050E00E940E26A881B9810D93ED
:102B10001C93A881B9810D911C9142E050E0040FF3
:102B2000151FA881B9810D931C93A5EDB0E00D91FF
:102B30001D912D913C91AEE7B0E04D915D916D916D
:102B40007C910E948F26A5EDB0E00D931D932D93EF
:102B50003D93A5EDB0E00D911D912D913C91A1E724
:102B6000B0E04D915C91662777270E948F26A5EDF6
:102B7000B0E00D931D932D933D930E94E51DA88118
:102B8000B981AD90BC90ADEDB0E0AA0DBB1D8C91AC
:102B9000AA81BB818D9388278D938D938C93A88177
:102BA000B9810E940125AA81BB810D911D912D91B2
:102BB0003C9140E051E060E070E00E941826AA815C
:102BC000BB810D931D932D933D93AA81BB810D91E4
:102BD0001D912D913C91A881B981AD90BC90ADED36
:102BE000B0E0AA0DBB1D4C915527662777270E94A0
:102BF0008F26AA81BB810D931D932D933D93009148
:102C000082000B3011F00C946516A881B9810E94E6
:102C10000125AA81BB810D911D912D913C9140E030
:102C200051E060E070E00E941826AA81BB810D93FC
:102C30001D932D933D93AA81BB810D911D912D91E3
:102C40003C91A881B981AD90BC90ADEDB0E0AA0DEA
:102C5000BB1D4C915527662777270E948F26AA8196
:102C6000BB810D931D932D933D93A881B9810E9443
:102C70000125AA81BB810D911D912D913C9140E0D0
:102C800051E060E070E00E941826AA81BB810D939C
:102C90001D932D933D93AA81BB810D911D912D9183
:102CA0003C91A881B981AD90BC90ADEDB0E0AA0D8A
:102CB000BB1D4C915527662777270E948F26AA8136
:102CC000BB810D931D932D933D93AA81BB810D91E3
:102CD0001D912D913C91AE81BF810D931D932D933C
:102CE0003C9386E0481A8827580A2496089580E085
:102CF000A881B9818C930027BB27A0E38C9183FB2B
:102D00000EF401E040E0041711F00C948B1682E001
:102D1000A881B9818C930027BB27A0E38C9184FB09
:102D20000EF401E040E0041711F00C949B1681E0D2
:102D3000A881B9818C930027BB27A3E38C9181FBE9
:102D40000EF401E040E0041711F00C94AB1683E0A0
:102D5000A881B9818C930027BB27A3E38C9181FBC9
:102D60000EF401E040E0041781E009F080E08F9369
:102D70000027BB27A0E38C9183FB0EF401E040E029
:102D8000041781E009F080E09F918923882311F4E2
:102D90000C94CE1684E0A881B9818C93089581E0CB
:102DA0000E94082681E00E9408265398549880E0EB
:102DB00081BB909A919AEF93FF93E0EFF1E00E942C
:102DC000CD25FF91EF9180E0AA81BB818C9300918A
:102DD0007000003081E009F080E08F930091700076
:102DE000023081E009F080E09F91892B882311F463
:102DF0000C94A2170027BB27A0E38C9180FB0EF454
:102E000001E040E0041711F00C940A1781E0AA8158
:102E1000BB818C930027BB27A0E38C9181FB0EF430
:102E200001E040E0041711F00C941B17AA81BB814C
:102E30008C918E5F8C930027BB27A9E38C9185FB37
:102E40000EF401E040E0041711F00C942C17AA8155
:102E5000BB818C918C5F8C930027BB27A9E38C915D
:102E600084FB0EF401E040E0041711F00C943D17D0
:102E7000AA81BB818C91885F8C93AA81BB810C91C4
:102E8000003018F011F00C9447170C94A0178AE04A
:102E900090E00E94F92580E0A881B9818C930027F9
:102EA000BB27A0E38C9180FB0EF401E040E0041707
:102EB00011F00C945F1781E0A881B9818C930027F1
:102EC000BB27A0E38C9181FB0EF401E040E00417E6
:102ED00011F00C947017A881B9818C918E5F8C933E
:102EE0000027BB27A9E38C9185FB0EF401E040E0AD
:102EF000041711F00C948117A881B9818C918C5F13
:102F00008C930027BB27A9E38C9184FB0EF401E08E
:102F100040E0041711F00C949217A881B9818C91AC
:102F2000885F8C93A881B9814C91AA81BB810C9157
:102F3000041711F40C94A01780E0AA81BB818C9334
:102F40000C9448180027BB27A0E38C9180FB0EF45B
:102F500001E041E0041711F00C94B21781E0AA815E
:102F6000BB818C930027BB27A0E38C9181FB0EF4DF
:102F700001E041E0041711F00C94C317AA81BB8152
:102F80008C918E5F8C930027BB27A9E38C9185FBE6
:102F90000EF401E041E0041711F00C94D417AA815B
:102FA000BB818C918C5F8C930027BB27A9E38C910C
:102FB00084FB0EF401E041E0041711F00C94E517D6
:102FC000AA81BB818C91885F8C93AA81BB810C9173
:102FD000003018F011F00C94EF170C9448188AE0A8
:102FE00090E00E94F92580E0A881B9818C930027A8
:102FF000BB27A0E38C9180FB0EF401E041E00417B5
:1030000011F00C94071881E0A881B9818C930027F6
:10301000BB27A0E38C9181FB0EF401E041E0041793
:1030200011F00C941818A881B9818C918E5F8C9343
:103030000027BB27A9E38C9185FB0EF401E041E05A
:10304000041711F00C942918A881B9818C918C5F18
:103050008C930027BB27A9E38C9184FB0EF401E03D
:1030600041E0041711F00C943A18A881B9818C91B1
:10307000885F8C93A881B9814C91AA81BB810C9106
:10308000041711F40C94481880E0AA81BB818C933A
:1030900000917000003081E009F080E08F93009192
:1030A0007000013081E009F080E09F91892B882336
:1030B00011F40C949E18AA81BB810C91033011F07D
:1030C0000C94681882E0AA81BB818C930C949E18A2
:1030D000AA81BB810C91043081E008F480E08F93D9
:1030E000AA81BB810C91073081E010F009F080E0EB
:1030F0009F918923882311F40C94841883E0AA817A
:10310000BB818C930C949E18AA81BB810C910830D2
:1031100081E008F480E08F93AA81BB810C910F308D
:1031200081E010F009F080E09F918923882311F459
:103130000C949E1884E0AA81BB818C9381E081BBB2
:103140009198539A549AAA81BB818C91AC81BD818C
:103150008C9382E0481A8827580A2496089581E0C3
:103160000E94082681E00E940826AC81BD818C91D6
:10317000A881B9818C930E94D50788EC90E00E94C9
:10318000F9255A924A9281E0A42DB52D8C9381E0C5
:103190000E94E7240E945722229681E00E94E324A5
:1031A000A895EBE6F0E0FA93EA930E947716229650
:1031B0008AE090E00E94F92500916B00003011F048
:1031C0000C94D01886E990E00E94F9255A924A9210
:1031D00080E0A42DB52D8C9381E00E94E7240E940D
:1031E0005722229681E00E94E32484E690E00E9428
:1031F000F9255A924A9280E0A42DB52D8C9381E056
:103200000E94E7240E945722229681E00E94E32434
:10321000A895EBE6F0E0FA93EA930E9477162296DF
:103220000E94D7075A924A9281E0A42DB52D8C9323
:1032300081E00E94E7240E945722229681E00E94AA
:10324000E32484E690E00E94F9255A924A9280E0B5
:10325000A42DB52D8C9381E00E94E7240E94572273
:10326000229681E00E94E3248AE090E00E94F92502
:103270005A924A9280E0A42DB52D8C9381E00E9451
:10328000E7240E945722229681E00E94E3240E94B4
:10329000D50786E990E00E94F92500916B00003087
:1032A00018F011F00C9456190C94081988E790E066
:1032B0000E94F9255A924A9281E0A42DB52D8C9353
:1032C00081E00E94E7240E946D1A229681E00E940C
:1032D000E324A881B9810C91023011F00C94B0194B
:1032E00000916B00013011F00C947B1981E0809308
:1032F000C5000C94A919023011F00C94931980E0C8
:103300008093C5005A924A9281E0A42DB52D8C93EA
:1033100081E00E94E7240E946D1A229681E00E94BB
:10332000E3240C94A919033011F00C94A91983E03B
:103330008093C5005A924A9282E0A42DB52D8C93B9
:1033400081E00E94E7240E946D1A229681E00E948B
:10335000E324EEE0F0E0A5ECB0E07BE70E9422275A
:10336000A881B9810C91033011F00C94D919009106
:103370006B00013011F00C94C21981E08093700051
:103380000C94D219023011F00C94CB1980E0809388
:1033900070000C94D219033011F00C94D21982E011
:1033A00080937000E1E1F0E0A0E7B0E07BE70E94ED
:1033B0002227A881B9810C91013011F00C942B1AAD
:1033C00000916B00013011F00C94F219A6ECB0E002
:1033D0008C91897F8C93A6ECB0E08C9182608C9369
:1033E0000C94241A023011F00C940C1AA6ECB0E0E4
:1033F0008C91897F8C935A924A9281E0A42DB52DAD
:103400008C9381E00E94E7240E946D1A229681E04D
:103410000E94E3240C94241A033011F00C94241A13
:10342000A6ECB0E08C9186608C935A924A9284E02C
:10343000A42DB52D8C9381E00E94E7240E946D1A83
:10344000229681E00E94E324EFE0F0E0A6ECB0E0F9
:103450007BE70E9422270E94D907A895EBE6F0E0BF
:10346000FA93EA930E947716229685E090E00E94F4
:10347000F92500916B00003011F00C942D1A86E9AB
:1034800090E00E94F9255A924A9280E0A42DB52D31
:103490008C9381E00E94E7240E945722229681E0CB
:1034A0000E94E32486E990E00E94F9255A924A920C
:1034B00080E0A42DB52D8C9381E00E94E7240E942A
:1034C0005722229681E00E94E3240E94D70782E0DF
:1034D000481A8827580A2496089581E00E940826F1
:1034E00081E0A881B9818C93AA81BB814C91A8818C
:1034F000B9810C91041718F011F00C949A1A5A9291
:103500004A9282E0A42DB52D8C9381E00E94E7249D
:103510000E945722229681E00E94E3248DE790E0EA
:103520000E94F925A881B9818C918F5F8C9310F44A
:103530000C94741A81E0481A8827580A2296089534
:1035400081E00E94082681E0A881B9818C93A8813E
:10355000B9810C91063018F011F00C94C31A0E9436
:10356000D5078FE090E00E94F9250E94D70784E6F6
:1035700090E00E94F925A881B9818C918F5F8C938E
:1035800010F40C94A71A81E0481A8827580A22964A
:1035900008950E94E525C39A88EC90E00E94F925E1
:1035A00081B5886081BD0E9419215A924A9281E0BA
:1035B000A42DB52D8C9381E00E94E7240E94652103
:1035C000229681E00E94E32481B5886181BD877FD6
:1035D00081BD84E690E00E94F925FF27E0E1FA939F
:1035E000EA935A924A928BE0A42DB52D8C9381E0F8
:1035F0000E94E7240E94ED23249681E00E94E324A8
:10360000013051E0150711F00C94191B5A924A929F
:10361000A0ECB0E08D919C91A42DB52D8D939C9341
:1036200082E00E94E7240E94FD21229682E00E940F
:10363000E3245A924A9282E3A42DB52D8C9381E023
:103640000E94E7240E946521229681E00E94E324E3
:10365000C29AD89A82E390E00E94F925089581E009
:103660000E94082681E00E9408268FEFAA81BB8174
:103670008C9380E0A881B9818C93A881B9810C9149
:10368000073018F011F00C94521B91E0AA81BB8115
:103690000E94DB25A881B9818C918F5F8C9310F4F7
:1036A0000C943D1B82E0481A8827580A24960895F6
:1036B00081E00E94082681E00E94082681E00E94A5
:1036C000082682E00E94082682E00E9408268FEFEA
:1036D000AA85BB858C9381E0A885B9858C93A88544
:1036E000B9850C91003418F011F00C94811B0E94E4
:1036F0002F1BA885B9858C918F5F8C9310F40C9447
:103700006F1BC49881E0A885B9858C93A885B9857D
:103710000C91003418F011F00C94981B0E942F1B90
:10372000A885B9858C918F5F8C9310F40C94861BBF
:103730008AE090E00E94F925A895EE81FF81FA9336
:10374000EA935A924A9280E4A42DB52D8C9381E09D
:103750000E94E7245A924A9200E010E020E030E014
:10376000A42DB52D0D931D932D933C9384E00E94C1
:10377000E7240E948E20269685E00E94E324AE81F5
:10378000BF810C91013011F40C94C91BC49A0C94A4
:10379000DF1D81E0AA85BB858C93A89580E090E031
:1037A000A881B9818D939C93EE81FF81FA93EA936E
:1037B0005A924A9281E4A42DB52D8C9381E00E9407
:1037C000E7245A924A9200E010E020E030E0A42D75
:1037D000B52D0D931D932D933C9384E00E94E72417
:1037E0000E948E20269685E00E94E324A881B9815C
:1037F0000E94FA24AE81BF810C91003081E009F073
:1038000080E08F93A881B9810D911C91003050E028
:10381000150781E009F080E09F91892B882311F43E
:103820000C94D41BC49AA881B9810D911C910030CD
:1038300050E0150711F00C941F1C0C94DF1DA89587
:1038400084E690E00E94F925A895C49881E090E074
:103850000E94F925EE81FF81FA93EA935A924A92E7
:1038600080E5A42DB52D8C9381E00E94E7245A9227
:103870004A9201E010E020E030E0A42DB52D0D9338
:103880001D932D933C9384E00E94E7240E948E2098
:10389000269685E00E94E32485E090E00E94F925C9
:1038A000C49A8AE090E00E94F925A89500E010E013
:1038B00020E030E0AEE7B0E00D931D932D933C93F4
:1038C00000E010E020E030E0A5EDB0E00D931D93A6
:1038D0002D933C930E94E51D00E010E020E030E0D5
:1038E000A5EDB0E00D931D932D933C930027ACE61E
:1038F000B0E08C9180FB0EF401E041E0041711F080
:103900000C94841C0C94DF1DA8950091EA000230F1
:1039100011F40C94181D8091A00280938200A7EAF4
:10392000B2E00D91112740E051E00E940E26AA81DD
:10393000BB810D931C93AA81BB810D911C91A6EABA
:10394000B2E04D915527040F151FAA81BB810D933D
:103950001C93AA81BB810D911C912227332740E043
:1039600050E061E070E00E941826AEE7B0E00D93F1
:103970001D932D933D93A5EAB2E00D91112740E0F0
:1039800051E00E940E26AA81BB810D931C93AA814F
:10399000BB810D911C91A4EAB2E04D915527040F13
:1039A000151FAA81BB810D931C93AEE7B0E00D916A
:1039B0001D912D913C91AA81BB814D915C9166270F
:1039C00077270E948F26AEE7B0E00D931D932D93CD
:1039D0003D93009182000C3011F00C94F21C8BE0AE
:1039E00080938200009182000E3011F00C94FB1C39
:1039F0008BE080938200009182000F3011F00C94D4
:103A0000041D8BE080938200AEE7B0E00D911D9124
:103A10002D913C91A5EDB0E00D931D932D933C931A
:103A20000E94E51DA5EDB0E00E9408250C942A1D1A
:103A300000911401063411F00C94211D84E0809350
:103A4000820000913001063411F00C942A1D8BE0A5
:103A5000809382008091EB0080937300009173004B
:103A6000003011F00C94361D0C94DF1D0091730092
:103A7000003418F011F00C943F1D0C94411D0C946F
:103A8000DF1D8091EC00AE81BF818C938091ED00B1
:103A9000AC81BD818C93AC81BD819C91AE81BF8195
:103AA0008C91A1E7B0E08D939C938091F400AE815E
:103AB000BF818C938091F500AC81BD818C93AC81EA
:103AC000BD819C91AE81BF818C91A4E7B0E08D93C4
:103AD0009C93A4E7B0E00D911C91003050E01507D5
:103AE00011F00C94891D80910201AE81BF818C93ED
:103AF00080910301AC81BD818C93AC81BD819C918F
:103B0000AE81BF818C91A4E7B0E08D939C930C941F
:103B1000891DA4E7B0E00D911C91003050E015071D
:103B200011F00C94951D0C94DF1D02E010E020E0D4
:103B300030E0A4E7B0E04D915C91662777270E94C2
:103B40001826A6E7B0E00D931D932D933D93A6E7AD
:103B5000B0E00D911D912D913C91A1E7B0E04D9108
:103B60005C91662777270E948F26A6E7B0E00D9329
:103B70001D932D933D93A6E7B0E00D911D912D91DE
:103B80003C91A5EDB0E04D915D916D917C910E94CD
:103B90008F26A6E7B0E00D931D932D933D93A6E7E6
:103BA000B0E00D911D912D913C91A5EDB0E00D93EC
:103BB0001D932D933C9380E0AA85BB858C9387E071
:103BC000481A8827580A2A96089581E00E940826F4
:103BD00081E00E94082682E00E94082682E00E947E
:103BE00008268FEFAE81BF818C9391E0AE81BF81BB
:103BF0000E94DB2591E0AE81BF810E94DB2591E030
:103C0000AE81BF810E94DB2591E0AE81BF810E9421
:103C1000DB2591E0AE81BF810E94DB2591E0AE8182
:103C2000BF810E94DB2591E0AE81BF810E94DB2530
:103C300091E0AE81BF810E94DB2591E0AE81BF8122
:103C40000E94DB2591E0AE81BF810E94DB2591E0DF
:103C5000AE81BF810E94DB2591E0AE81BF810E94D1
:103C6000DB2591E0AE81BF810E94DB2591E0AE8132
:103C7000BF810E94DB2591E0AE81BF810E94DB25E0
:103C800091E0AE81BF810E94DB25C49880E090E086
:103C9000A881B9818D939C938FEF0E94EC250E949F
:103CA000EE250E94ED25AE81BF818C93A881B9815C
:103CB0000E94FA24AE81BF810C91003081E009F4AA
:103CC00080E08F93A881B9810D911C91003050E064
:103CD000150781E009F080E09F91892B882311F47A
:103CE0000C944C1EA881B9810D911C91003050E0BC
:103CF000150711F00C94831E80916C0081608093F5
:103D00006C000C94A81FEE81FF81FA93EA935A92FB
:103D10004A9281E5A42DB52D8C9381E00E94E72481
:103D20005A924A92A5EDB0E00D911D912D913C91D2
:103D3000A42DB52D0D931D932D933C9384E00E94EB
:103D4000E7240E948E20269685E00E94E324002727
:103D5000ACE6B0E08C9180FB0EF401E041E004178A
:103D600011F00C94B51E0C94A81FA895AE81BF81CC
:103D70000C91003011F00C94FA1E80E090E0A881C4
:103D8000B9818D939C938FEF0E94EC250E94EE25C4
:103D90000E94ED25AE81BF818C93A881B9810E94DC
:103DA000FA24AE81BF810C91003081E009F480E0FB
:103DB0008F93A881B9810D911C91003050E01507B7
:103DC00081E009F080E09F91892B882311F40C9405
:103DD000C31EA881B9810D911C91003050E01507D8
:103DE00011F00C94FA1E80916C00816080936C003D
:103DF0000C94A81FAE81BF810C910F3F11F00C9461
:103E00003E1F80E090E0A881B9818D939C938FEF55
:103E10000E94EC250E94EE250E94ED25AE81BF8117
:103E20008C93A881B9810E94FA24AE81BF810C9144
:103E30000F3F81E009F480E08F93A881B9810D9153
:103E40001C91003050E0150781E009F080E09F915F
:103E5000892B882311F40C94071FA881B9810D9137
:103E60001C91003050E0150711F00C943E1F80911A
:103E70006C00816080936C000C94A81FAE81BF81A0
:103E80000C910E3F11F40C944D1FC49A80916C005C
:103E9000816080936C000C94A81F80E090E0AA8160
:103EA000BB818D939C9380E0AE81BF818C93AE816A
:103EB000BF810C910F3F18F011F00C948F1FAA8155
:103EC000BB810E94FA248FEF0E94EC250E94EE2510
:103ED0000E94ED25AA81BB81AD90BC90ADEDB0E014
:103EE000AA0DBB1D8C93AA81BB810E94FA248FEF7F
:103EF0000E94EC250E94EE250E94ED25AA81BB813F
:103F0000AD90BC90ADEDB0E0AA0DBB1D8C93AE8121
:103F1000BF818C918F5F8C9310F40C94571F8FEF9F
:103F20000E94EC250E94EE250E94ED25AE81BF8106
:103F30008C938FEF0E94EC250E94EE250E94ED25C8
:103F4000AE81BF818C93C49AA5EDB0E00E94EB24B2
:103F500086E0481A8827580A2896089582E00E9429
:103F6000082681E00E94082680E0AE81BF818C9304
:103F70000E942F1BC49880E090E0AA81BB818D93A2
:103F80009C938FEF0E94EC250E94EE250E94ED2568
:103F9000A881B9818C93AA81BB810E94FA24A8814F
:103FA000B9810C91003081E009F480E08F93AA81FF
:103FB000BB810D911C91003050E0150781E009F0A4
:103FC00080E09F91892B882311F40C94C11FAA8152
:103FD000BB810D911C91003050E0150711F00C943D
:103FE000F81F80916C00816080936C000C94882095
:103FF000E881F981FA93EA935A924A9281E5A42DD5
:10400000B52D8C9381E00E94E7245A924A92AA85AA
:10401000BB850D911D912D913C91A42DB52D0D9336
:104020001D932D933C9384E00E94E7240E948E20F0
:10403000269685E00E94E324A881B9810C91003086
:1040400011F00C944F2080E090E0AA81BB818D9309
:104050009C938FEF0E94EC250E94EE250E94ED2597
:10406000A881B9818C93AA81BB810E94FA24A8817E
:10407000B9810C91003081E009F480E08F93AA812E
:10408000BB810D911C91003050E0150781E009F0D3
:1040900080E09F91892B882311F40C942920A8811A
:1040A000B9810C910F3F11F00C94822080E090E0D8
:1040B000AA81BB818D939C938FEF0E94EC250E9477
:1040C000EE250E94ED25A881B9818C93AA81BB8140
:1040D0000E94FA24A881B9810C910F3F81E009F474
:1040E00080E08F93AA81BB810D911C91003050E03C
:1040F000150781E009F080E09F91892B882311F456
:104100000C945C20A881B9818C91AE81BF818C9385
:1041100083E0481A8827580A2496089584E00E946C
:10412000082681E00E94082682E00E9408268FEF80
:10413000AA81BB818C9391E0AA81BB810E94DB257F
:1041400091E0A885B9850E94DB25AE81BF810D91E4
:104150001D912D913C9140E052E060E070E00E94A2
:104160001826AC81BD810D931D932D933D93AC8199
:10417000BD818F9314968E910E940E218E910E9484
:104180000E218E910E940E218E910E940E2185E9B2
:104190000E940E218F9180E090E0A881B9818D93DB
:1041A0009C938FEF0E94EC250E94EE250E94ED2546
:1041B000AA81BB818C93A881B9810E94FA24AA812B
:1041C000BB810C910F3F81E009F480E08F93A881BF
:1041D000B9810D911C91003050E0150781E009F084
:1041E00080E09F91892B882311F40C94D120A88121
:1041F000B9810D911C91003050E0150711F00C941D
:10420000062180916C00816080936C00AA81BB8143
:104210008C91AA85BB858C930C9413218FB9779BC5
:10422000FECF8FB1089587E0481A8827580A26964E
:1042300008955A924A9284E298E0A42DB52D8D9368
:104240009C9382E00E94E7245A924A9280E0A42D37
:10425000B52D8C9381E00E94E7240E94922324963E
:1042600083E00E94E324EF93FF93ECE8F1E00E94E7
:10427000CD25FF91EF91BB27A0E38C9182FBDEF768
:1042800089E190E00E94F9255A924A9280E298E0F2
:10429000A42DB52D8D939C9382E00E94E7245A9221
:1042A0004A9280E0A42DB52D8C9381E00E94E724F2
:1042B0000E949223249683E00E94E32489E190E007
:1042C0000E94F9250E941A22089582E00E94082681
:1042D00000E011E0AA81BB814D9155270E940E2676
:1042E000A881B9810D931C93A881B9810D911C916E
:1042F000AA81BB814D915527040F151FA881B98153
:104300000D931C935A924A92AA81BB818D919C91E4
:10431000A42DB52D8D939C9382E00E94E7245A92A0
:104320004A928BE0A42DB52D8C9381E00E94E72466
:104330000E949223249683E00E94E3245A924A9298
:1043400080E298E0A42DB52D8D939C9382E00E948D
:10435000E7245A924A9280E0A42DB52D8C9381E0F7
:104360000E94E7240E949223249683E00E94E32483
:1043700082E0481A8827580A2296089582E00E940F
:10438000082600E110E0AC81BD814D9155270E94C7
:104390000E26A881B9810D931C93A881B9810D9136
:1043A0001C91AA81BB814D915527040F151FA8812F
:1043B000B9810D931C935A924A92AA81BB818D9127
:1043C0009C91A42DB52D8D939C9382E00E94E724AF
:1043D0005A924A9282E0A42DB52D8C9381E00E94DE
:1043E000E7240E949223249683E00E94E32482E043
:1043F000481A8827580A229608955A924A92AA8102
:10440000BB818D919C91A42DB52D8D939C9382E0C1
:104410000E94E7245A924A9283E0A42DB52D8C93F2
:1044200081E00E94E7240E949223249683E00E9468
:10443000E324089581E00E94082681E00E94082676
:10444000C49AD898C29880E0A881B9818C9380E002
:10445000AA81BB818C93AA81BB810C910F3118F08A
:1044600011F00C944F2291E0A881B9810E94DB25C4
:1044700091E0A881B9810E94DB2591E0A881B981F2
:104480000E94DB2591E0A881B9810E94DB25AA81E9
:10449000BB818C918F5F8C9310F40C942B22C29A69
:1044A000D89A82E0481A8827580A2496089581E00D
:1044B0000E9408265A924A9280E298E0A42DB52DD7
:1044C0008D939C9382E00E94E7245A924A9280E066
:1044D000A42DB52D8C9381E00E94E7240E949223A5
:1044E000249683E00E94E324AA81BB810C910030D2
:1044F00011F00C948A225A924A9280E0A42DB52D94
:104500008C9381E00E94E7240E940423229681E09C
:104510000E94E324AA81BB810C91013011F00C941C
:10452000A0225A924A9285E6A42DB52D8C9381E063
:104530000E94E7240E940423229681E00E94E32443
:10454000AA81BB810C91023011F00C94CD225A92B9
:104550004A9283E6A42DB52D8C9381E00E94E72436
:104560000E940423229681E00E94E32488EC90E0DC
:104570000E94F9255A924A9280E0A42DB52D8C9381
:1045800081E00E94E7240E940423229681E00E9499
:10459000E32482E390E00E94F925AA81BB810C917B
:1045A000033011F00C94F6225A924A9282E6A42D1E
:1045B000B52D8C9381E00E94E7240E94042322966B
:1045C00081E00E94E32480E991E00E94F9255A925B
:1045D0004A9280E0A42DB52D8C9381E00E94E724BF
:1045E0000E940423229681E00E94E3248AE090E066
:1045F0000E94F9258AE090E00E94F92581E0481A9E
:104600008827580A2296089581E00E940826C49AB5
:10461000D898C298AA81BB810C91003018F011F093
:104620000C9414230C944E2383E5A881B9818C93B8
:1046300091E0A881B9810E94DB258FEEA881B98124
:104640008C9391E0A881B9810E94DB258EE6A88138
:10465000B9818C9391E0A881B9810E94DB2591E01A
:10466000AA81BB810E94DB2580E0A881B9818C935F
:1046700091E0A881B9810E94DB2591E0A881B981F0
:104680000E94DB2591E0A881B9810E94DB2591E0A1
:10469000A881B9810E94DB250C948A2385E4A88136
:1046A000B9818C9391E0A881B9810E94DB2588E7CC
:1046B000A881B9818C9391E0A881B9810E94DB2502
:1046C00089E6A881B9818C9391E0A881B9810E9483
:1046D000DB2584E7A881B9818C9391E0A881B98119
:1046E0000E94DB2580E0A881B9818C9391E0A881AC
:1046F000B9810E94DB2591E0A881B9810E94DB2568
:1047000091E0A881B9810E94DB2591E0A881B9815F
:104710000E94DB25C29AD89A81E0481A8827580A55
:104720002296089581E00E940826C29AD8985A924B
:104730004A9282E0A42DB52D8C9381E00E94E7245B
:104740000E944724229681E00E94E3245A924A92D2
:10475000AC81BD818C91A42DB52D8C9381E00E94FC
:10476000E7240E944724229681E00E94E324AC8142
:10477000BD8111968C91A881B9818C935A924A92ED
:10478000AA81BB818C91A42DB52D8C9381E00E94D0
:10479000E7240E944724229681E00E94E324AC8112
:1047A000BD818C91A881B9818C935A924A92AA8139
:1047B000BB818C91A42DB52D8C9381E00E94E724C0
:1047C0000E944724229681E00E94E324D89A81E047
:1047D000481A8827580A2296089581E00E940826E0
:1047E00081E00E94082682E00E940826C29AD8989A
:1047F0005A924A9283E0A42DB52D8C9381E00E94B9
:10480000E7240E944724229681E00E94E3245A92E2
:104810004A92A885B9858C91A42DB52D8C9381E001
:104820000E94E7240E944724229681E00E94E3240C
:10483000EC81FD81FA93EA930E944D242296EA814D
:10484000FB81FA93EA930E944D242296D89AAC8178
:10485000BD810D91112740E051E00E940E26A881F4
:10486000B9810D931C93A881B9810D911C91AA81E6
:10487000BB814D915527040F151FA885B9850D9350
:104880001C9384E0481A8827580A2696089591E0D8
:10489000A881B9810E94DB25089581E00E94082645
:1048A00091E0A881B9810E94D025A881B9818C911D
:1048B000AA81BB818C9381E0481A8827580A2296E6
:1048C000089582E00E94082681E00E940826C49A8A
:1048D000BB27A0E38C9182FBDEF7C298AC81BD813F
:1048E0000D911C91003052E0150711F00C94B0248A
:1048F00081E090E0AA81BB818D939C9380E0A881A8
:10490000B9818C93A881B9810C910F3018F011F006
:104910000C94AE24BB27A0E38C9182FBDEF790E2DF
:10492000AA81BB81AD90BC90ADEDB0E0AA0DBB1DDE
:104930000E94DB25AA81BB810D911C9140E250E0D1
:10494000040F151FAA81BB810D931C93A881B98107
:104950008C918F5F8C9310F40C9482240C94DC2443
:1049600081E090E0AA81BB818D939C93AC81BD8155
:104970004D915C91AA81BB810D911C910417150783
:1049800018F011F00C94DC24BB27A0E38C9182FB7F
:10499000DEF7C29A91E0AA81BB81AD90BC90ADEDEB
:1049A000B0E0AA0DBB1D0E94DB25AA81BB810E943D
:1049B000FA2410F40C94B624C29A83E0481A88278B
:1049C000580A24960895481A8827580A0895480EC8
:1049D0008827581E08950D911D912D913C9181E0DD
:1049E000080F8827181F281F381F3C932E931E93EB
:1049F0000E930895ED91FC91EF5FFF4FFC93EE93C2
:104A00000895ED91FC91E150F040FC93EE930895F0
:104A10000D911D912D913C9101501040204030404E
:104A20003C932E931E930E9308954091DF02509174
:104A3000E0020DE815E30E94292549E156E3040F41
:104A4000151F0093DF021093E002498158810C94F6
:104A50004F2509D00E940E2600FC10D0089503D0E7
:104A60001ED001F8F9CF0024E89457FF02C009D006
:104A7000689400F80BD010F80124089502D009D0F2
:104A80000895509540954F5F5F4F0895E89417FF44
:104A90000895009510950F5F1F4F68940895352F66
:104AA000242FE894452B11F468940895512F402F3A
:104AB0000027112780E1440F551F001F111F021B03
:104AC000130B416018F4020F131F4E7F8A9599F75C
:104AD00008958F938D918823E9F711978F91089509
:104AE00088EE93E086D03197D9F7089500FC05D081
:104AF000089530D005D001F8F9CF37D03FD00895D0
:104B0000842F952FA62FB72FE894452B462B472BA4
:104B100011F468940895402F512F622F732F0027AE
:104B2000112722273327F0E2440F551F661F771FF6
:104B3000001F111F221F331F081B190B2A0B3B0BD1
:104B4000416028F4080F191F2A1F3B1F4E7FFA955A
:104B500059F708950024E89477FF02C006D06894BE
:104B600000F809D010F80124089512D04F5F5F4F6C
:104B70006F4F7F4F0895E89437FF08950095109583
:104B8000209530950F5F1F4F2F4F3F4F689408952A
:104B9000409550956095709508953197F1F7089577
:104BA0000E94EC258C910E94EE258D939A95D1F769
:104BB0000E94ED2508950E94EC258D910E94EE251E
:104BC0009A95D9F70E94ED250895BF9ABE98C69A86
:104BD000BD9A80E58DB90895089508958FB9779BA2
:104BE000FECF8FB10895689462F80895E89462F852
:104BF0000895EF93FF93EE27E82BE92B31F0E0EDDA
:104C0000F7E03197F1F70197D1F7FF91EF91089510
:104C10005A924A92480E8827581E08950F92B8015A
:104C2000469F8001479F100D569F100D0F900895CD
:104C30000F921F922F92C801D901489F80014A9F6D
:104C400090014B9F202C499F100D211D321D5A9F12
:104C5000202C589F100D211D321D599F200D311DF4
:104C6000689F200D311D699F300D789F300D2F906A
:104C70001F900F9008950E9441260D920020D9F7B1
:104C80000895C895319600200895819104D08D93A0
:104C90008823D9F70895813618F08B3708F48F7D73
:104CA00008952E2E3F2E992781918D3209F09395EC
:104CB0008823D1F79A95E22DF32D112361F009177E
:104CC00018F011F0101B01C0191B28F021F080E230
:104CD0008D931A95E9F780818D3219F48D93319671
:104CE00004C0222311F08BE28D93091738F031F0C4
:104CF000091B21F080E38D930A95E9F781918D934B
:104D00008823E1F7332351F0EA2FFB2F31963395B7
:104D10008E9182933A95E1F78EE28C930895040F79
:104D2000151F261F371F0895041B150B260B370B65
:104D3000089504171507260737070895000F111F58
:104D4000221F331F089500951095209530950F5F11
:104D50001F4F2F4F3F4F0895019110810EC00191B9
:104D60001191219130810BC00191108117FF05C075
:104D70003FEF2FEF04C0008111272227332737FF91
:104D800003C0E1DF8DE28D93CF93DF93CF92DF926B
:104D9000EF92AA24BB24CC24DD24EE2440E2CAE016
:104DA000DD2755E093E38881890F87FD9F7083FDA0
:104DB000907F891B89935A95A9F7C0DFAA1CBB1C59
:104DC000CC1CDD1CEE1C4A9551F7E894EFE0FF2760
:104DD00082910ED0EB30E0F71EF068948A2D0CD053
:104DE00088278D93EF90DF90CF90DF91CF9108953A
:104DF000982F829501D0892F8F70805D26F08033A7
:104E000009F4089568948D93089588278D930895E3
:104E100081918D938823E1F70895099191919923C8
:104E200051F08A95D9F7319781918D930A9519F0B0
:104E30008823D1F70895E9CFE199FECFEEBBFFBB00
:104E40003196089591E001C092E07B3751F47FB72D
:104E5000F894F2DF8D918DBBE29AE19A9A95C9F7A9
:104E60007FBF7727089591E001C092E0E5DFE09AE7
:104E70008DB38D939A95D1F70895FF93881BF9E030
:104E8000001FFA9511F4FF910895881F841B18F4F0
:104E9000840F8894F5CF0894F3CF689401C0E89408
:104EA000AF93BF938D9116F0919103C00E9441265C
:104EB000902D891718F011F48823A1F7BF91AF91B5
:104EC00008954F005A00590048004200434F4E4693
:064ED000494700002E001E
:00000001FF
